:020000040000FA
:02000000722864
:08000800F000030E8301F1007A
:100010000A08F2008A010408F3008A150A12002176
:1000200083017308840072088A00710E8300F00E49
:10003000700E0900A7002130A70700308A002708AA
:1000400082002034473448345334313435346334F7
:100050006C346F3463346B342034563431342E3482
:100060003034A7003830A70700308A002708820004
:1000700020344E346F34773420347734613469342B
:10008000743469346E346734A7004B30A7070030EE
:100090008A00270882006434653473346934673415
:1000A0006E34203432343034303434344A3475349D
:1000B0006E3431343034A7006230A70700308A0034
:1000C00027088200203462347934203454342E34AA
:1000D00048346134793461346D3469347A34753438
:1000E000203420348B13013090000B309700053002
:1000F0009600DC30950083168F30810006309F001B
:10010000850101308600E0308700203098004030C3
:1001100099000C15831290309800850186018701A3
:10012000203084008001840A71300402031D92286B
:10013000A030840020308000840AEF300402031DC8
:100140009A28912164008E018F01D0308B0080307D
:100150004321A10121081A205F21A10A2108103C96
:10016000031DAA28C0304321A101210831205F21AD
:10017000A10A21080C3C031DB5280712C321473CE6
:10018000031DBE28C321473C031DBE28C321413C9B
:10019000031DBE28C3212C3C031DBE28A0308400B3
:1001A000CE21031DD028A6308400CE21031DD528E2
:1001B000AF308400CE21031DDA28B0308400CE2178
:1001C000031DDF28BA308400CE21031DE428BB3094
:1001D0008400CE21031DE928BC308400CE21031DFC
:1001E000EE28BE30840020308000840AD53004021E
:1001F000031DF328BE308400CE21031DFC28C2302D
:100200008400CE21031D0129C321C321C9308400EC
:10021000CE21031D08296400C321523C031D0C2973
:10022000C3214D3C031D0C29C3214D3C031D0C294A
:10023000C3212C3C031D0C29CF3084000408D53C7D
:1002400003192529CE21031D1E296400BB3084001B
:100250000008A100313C031933292108323C03195D
:100260003329A01235292016A016201EBE282D08DD
:10027000031D3C29DC21BE28A100A10B4129362207
:10028000BE28B322BE28AB00F039A200A20E070898
:10029000F0392204870005128511851600008512A9
:1002A0002B080F39A2000708F039220487008516B1
:1002B0000000851278210800013043210800AB00BE
:1002C000F039A200A20E0708F039220487000512B7
:1002D00085158516000085122B080F39A200070826
:1002E000F039220487008516000085127821080065
:1002F000AB018316AF308700831285110516851672
:10030000070E8512F039AB008516070885120F39E4
:10031000AB04AB1B782905128316A030870083122B
:100320000800DD22F0300705F3388700051285113B
:10033000851600008512DD22F0300705F3388700AE
:1003400005128511851600008512D622F0300705AA
:10035000F338870005128511851600008512D62214
:10036000F0300705F2388700051285118516000068
:100370008512D6222C304321083043210C304321F2
:100380000630432108008C1EC32918193014981C0C
:10039000CC2918121816B0141A080800C321A1009D
:1003A0002C3C0319080021088000840A031108006E
:1003B0000C1ED829990008005C2180304321A03010
:1003C000840000085F21840AA4300402031DE1298F
:1003D00085304321B030840000085F21840ABA30A0
:1003E0000402031DEC298F304321BA308400000839
:1003F000A01E58305F21C0304321C2308400000865
:10040000203C03191E2A840A00082E3C03190D2AD9
:100410000408C93C03191E2A032AC330A100432142
:1004200084030408C13C03191E2A00085F21A103AC
:100430002108BF3C03191E2A21080F2AC43043217A
:100440006D305F21C6304321A630840000085F2153
:10045000840AAF300402031D262ACF304321AF3077
:1004600084000008A01E58305F2108005C21803005
:10047000432147305F21C93084000008203C031924
:100480005C2A840A00082E3C03194B2A0408CF3C3E
:1004900003195C2A412A8330A10043218403040804
:1004A000C83C03195C2A00085F21A1032108803C95
:1004B00003191E2A21084D2A843043216D305F2103
:1004C00020305F2153305F2161305F2174305F2124
:1004D000BC30840000085F21840ABE300402031D82
:1004E0006A2A20305F2148305F2144305F21BE30CE
:1004F00084000008203C0319932ABF3084000008C0
:100500002E3C031D8A2A8F304321BE308400000810
:100510005F21932A8E304321BE30840000085F2182
:10052000840A00085F21C0304321CF3084000008D6
:100530005F21840AD5300402031D972A20305F21F1
:1005400047305F2148305F2153305F2131305F21D8
:1005500035305F2176305F2131305F212E305F21D1
:1005600030305F2108005C2180304321A101210847
:1005700044205F21A10A2108103C031DB72AC03086
:100580004321A10121085B205F21A10A2108103C21
:10059000031DC22ACB2A000008000F30A400CA2283
:1005A000A40BCF2AD32AD42A000008000330A500C8
:1005B000CD22DA2AA50BD82A08009630A500CD2234
:1005C000A50BDF2A08001430A600DD22A60BE52AC1
:0205D000080021
:10100000A8000730A80708308A002808820040346A
:1010100079342434303419341234023478340034BE
:101020001034083403344634213406340E34273463
:101030000B340934713447342B3423340C342F34BB
:0E1040004E3463344134113477343F347F34FE
:101200008B184B210C1906218A0108000C11871E2E
:101210000B297C210C29AE010130AC070318B10A5F
:10122000201C1F29B20B1929B30B192920100712F2
:10123000252907162C1C05112C180515252906181B
:101240002529AC1C0511AC180515A01A2C2931193B
:101250002C29051485144729A01D3329AC194729C9
:10126000051485143F29AC1D4729051485142A0847
:101270001F390020A300230D860085104729290867
:101280001F390020A300230D860005104729A01553
:10129000AC1DA01108008B10201A5029071208005D
:1012A0002010A43084000008353C031D6029840A06
:1012B0000008393C031D60292014B2010430B3003A
:1012C000A5308400000AA3000F390A3C031D7329CE
:1012D000A901201C6D29AA010800A4308400000A7D
:1012E0000F39AA00080023080F39A900A430840090
:1012F00000080F39AA000800AE0A40302E02031978
:101300008629031C0800F030AE000800AD0A2D0845
:08131000033C0319AD010800C4
:02400E00763FFB
:00000001FF
